:100000000C9434000C9451000C9451000C94510049
:100010000C9451000C9451000C9451000C94E50088
:100020000C9451000C9451000C9451000C94B400A9
:100030000C9451000C9451000C9483000C945100CA
:100040000C9451000C9451000C9451000C945100EC
:100050000C9451000C9451000C9451000C945100DC
:100060000C9451000C94510011241FBECFEFD8E026
:10007000DEBFCDBF11E0A0E0B1E0E6EAF5E002C0EE
:1000800005900D92A231B107D9F711E0A2E1B1E0DC
:1000900001C01D92A731B107E1F70E9443010C9402
:1000A000D1020C9400008230910561F083309105FB
:1000B00099F00197C9F416BC80916E00826080931C
:1000C0006E0016C0109285001092840080916F001F
:1000D000826080936F000CC01092B200809170001B
:1000E00082608093700004C081E090E00E94D102A1
:1000F00078949FB7F894809114019FBF8823C9F327
:100100001092140108951F920F920FB60F921124AE
:100110002F933F938F939F9380911201909113019E
:100120000196909313018093120180911401813004
:1001300091F020911201309113018091150190915D
:1001400016012817390738F081E0809314011092C6
:100150001301109212019F918F913F912F910F9057
:100160000FBE0F901F9018951F920F920FB60F920F
:1001700011242F933F938F939F938091120190911D
:100180001301019690931301809312018091140141
:10019000813091F02091120130911301809115016D
:1001A000909116012817390738F081E080931401E7
:1001B00010921301109212019F918F913F912F91F4
:1001C0000F900FBE0F901F9018951F920F920FB6B1
:1001D0000F9211242F933F938F939F93809112013D
:1001E00090911301019690931301809312018091D5
:1001F0001401813091F0209112013091130180910E
:100200001501909116012817390738F081E0809385
:10021000140110921301109212019F918F913F913E
:100220002F910F900FBE0F901F901895FC01A1E821
:10023000B0E08C918D608C9322E030E03387228790
:10024000219AA0E8B0E08C9181688C93A8E8B0E096
:1002500011961C921E921C92B587A48785B5836067
:1002600085BD81E090E097878687309316012093C3
:10027000150124B5226024BD29EF27BD918B808B09
:1002800080E090E00895CF92DF92EF92FF92CF93BB
:1002900080E091E00E941601C12CD12C760160E033
:1002A00070E0CB01CEE16093000170930101809377
:1002B00002019093030180911001909111010E941D
:1002C0005300E0910C01F0910D01C0838FEFC81A2B
:1002D000D80AE80AF80AC701B6010E94E0012FE631
:1002E00032E143E05BE30E946E0220E030E0A901CE
:1002F0000E947C01D8CF5058BB27AA270ED0B4C08B
:10030000A5D030F0AAD020F031F49F3F11F41EF4B4
:100310009AC00EF4E095E7FB90C0E92FB6D080F3C9
:10032000BA17620773078407950718F071F49EF5F2
:10033000CEC00EF4E0950B2EBA2FA02D0B01B90103
:1003400090010C01CA01A0011124FF27591B99F04B
:10035000593F50F4503E68F11A16F040A22F232F57
:10036000342F4427585FF3CF469537952795A795A7
:10037000F0405395C9F77EF41F16BA0B620B730B4E
:10038000840BBAF09150A1F0FF0FBB1F661F771FBF
:10039000881FC2F70EC0BA0F621F731F841F48F474
:1003A000879577956795B795F7959E3F08F0B3CFFA
:1003B0009395880F08F09927EE0F979587950895E4
:1003C000E89409C097FB3EF49095809570956195EF
:1003D0007F4F8F4F9F4F9923A9F0F92F96E9BB27A5
:1003E0009395F695879577956795B795F111F8CF21
:1003F000FAF4BB0F11F460FF1BC06F5F7F4F8F4F8C
:100400009F4F16C0882311F096E911C0772321F081
:100410009EE8872F762F05C0662371F096E8862F19
:1004200070E060E02AF09A95660F771F881FDAF770
:10043000880F9695879597F9089597F99F6780E8B3
:1004400070E060E008959FEF80EC089500240A9426
:100450001616170618060906089500240A9412169F
:100460001306140605060895092E0394000C11F4D2
:10047000882352F0BB0F40F4BF2B11F460FF04C07F
:100480006F5F7F4F8F4F9F4F089557FD9058440FD8
:10049000551F59F05F3F71F04795880F97FB991FE3
:1004A00061F09F3F79F087950895121613061406A0
:1004B000551FF2CF4695F1DF08C01616170618062D
:1004C000991FF1CF86957105610508940895E89408
:1004D000BB2766277727CB0197F908950BD0C4CFA8
:1004E000B5DF28F0BADF18F0952309F0A6CFABCF1F
:1004F0001124EECFCADFA0F3959FD1F3950F50E002
:10050000551F629FF001729FBB27F00DB11D639FC5
:10051000AA27F00DB11DAA1F649F6627B00DA11D6B
:10052000661F829F2227B00DA11D621F739FB00D11
:10053000A11D621F839FA00D611D221F749F332781
:10054000A00D611D231F849F600D211D822F762F1A
:100550006A2F11249F5750408AF0E1F088234AF017
:10056000EE0FFF1FBB1F661F771F881F9150504063
:10057000A9F79E3F510570F060CFAACF5F3FECF323
:10058000983EDCF3869577956795B795F795E7954F
:100590009F5FC1F7FE2B880F911D9695879597F960
:0605A0000895F894FFCF5E
:1005A6000000000000006F12033B00000000000086
:0205B600000043
:00000001FF
